:100000000C9417060C94FE280C942B290C943F0694
:100010000C943F060C94BD0C0C943F060C943F06C8
:100020000C943F060C943F060C943F060C943F063C
:100030000C943F060C943F060C943F060C943F062C
:100040000C9458290C943F060C94122D0C944D2DB1
:100050000C943F060C943F060C943F060C943F060C
:100060000C943F060C943F065C1C631C631C5C1CD8
:10007000631C631C631C631C631C631C631C631C88
:10008000631C631C631C631C631CD11B631C631C0B
:10009000631C631C631C341B631C631C631C631C98
:1000A000631C631C631C631C631C631C631C631C58
:1000B000631C631C631CDD1BDD1BDD1BDD1BDD1BEB
:1000C000DD1BDD1BDD1BDD1B631C631C631C631C54
:1000D000631C631C391BDC1BDC1BDC1BDC1B631C73
:1000E000ED1BF51BFD1B051C0D1C151C1D1C251CEB
:1000F0002F1C391C431C4D1C801B401B631C631CA4
:10010000631C631CD11B631C631C631C631C631C8A
:10011000631C631C631CDB1BDB1BDB1BDB1B631C0B
:10012000ED1BF51BFD1B051C0D1C151C1D1C251CAA
:100130002F1C391C431C4D1C801B401B631C631C63
:10014000631C631CD11B941C941C941C941C941C55
:10015000941C941C941C941C941C941C941C941C1F
:10016000B41DB41DB41DB41DB41DB41DDB1CE51CB1
:10017000EF1CF91C5F1D691D771D881D251E951E2E
:10018000661E6B1E701E751E7A1E7F1E841E951EB7
:100190008F1E9A25AF25BB25C425D125F725FF2520
:1001A00022260F26456E746572206D656E752E2EA3
:1001B0002E00546F67676C6564206D6963726F50C1
:1001C000504D00546F67676C656420696E76657288
:1001D0007465642050504D2100546F67676C6564EE
:1001E000205458206D7574696E672100546F6767DD
:1001F0006C65642074656C656D657472792100505E
:10020000726F746F636F6C206572726F72207769A2
:1002100074682052580054696D656F757420776852
:10022000656E20636F6E6E656374696E6720746FB0
:1002300020525800507265737320616E79206B658F
:100240007920746F2063616E63656C00436F6E6E1E
:10025000656374696E6720746F2052582C20706F2C
:100260007765722075702074686520525820287751
:100270006974682062696E6420706C7567206966B5
:10028000206E6F74207573696E6720616C77617979
:10029000732062696E642900546F67676C6564201F
:1002A00027696D6D656469617465206F757470751B
:1002B000742700546F67676C65642027736C6176E0
:1002C00065206D6F64652700546F67676C656420F7
:1002D00027616C776179732062696E642700546FBF
:1002E00067676C65642050504D206368616E6E6571
:1002F0006C206C696D6974005365742052535349C6
:1003000020696E6A656374696F6E206368616E6EE2
:10031000656C2028303D3D64697361626C6529001D
:100320005365742050504D206D696E696D756D2058
:1003300073796E630053657420626561636F6E202C
:10034000696E74657276616C0053657420626561D4
:10035000636F6E2064656C6179005365742062651B
:1003600061636F6E206672657175656E6379206971
:100370006E20487A3A20303D64697361626C652C66
:100380002050783D504D52206368616E6E656C2040
:10039000782C2046783D465253206368616E6E6526
:1003A0006C2078005365742050574D2073746F7023
:1003B0002064656C61792028302064697361626C07
:1003C00065642C20312D323535203D3D20302E31D5
:1003D00073202D2035306D696E29005365742050CF
:1003E000504D2073746F702064656C6179202830E3
:1003F0002064697361626C65642C20312D3235355F
:10040000203D3D20302E3173202D2035306D696E1A
:100410002900536574206661696C736166652064A8
:10042000656C61792028302064697361626C656451
:100430002C20312D323535203D3D20302E3173209A
:100440002D2035306D696E29002A2A2A2A2A2A2A67
:100450002A2A2A2A2A2A2A2A2A2A2A2A2A2A2A2AFC
:100460002A2A2A2A2A2A0052582041636B656420CE
:100470002D2072657665727420737563636573737E
:1004800066756C21002A2A2A2A2A2A2A2A2A2A2A36
:100490002A2A2A2A2A2A2A2A2A2A2A2A2A2A2A2ABC
:1004A0002A2A002A2A2A2A2A2A2A2A2A2A2A2A2AD6
:1004B0002A2A2A2A2A2A2A2A2A2A2A2A2A2A2A2A9C
:1004C0000052582041636B6564202D207570646173
:1004D0007465207375636365737366756C21002A98
:1004E0002A2A2A2A2A2A2A2A2A2A2A2A2A2A2A2A6C
:1004F0002A2A2A2A2A2A2A2A2A2A2A2A0056616CE1
:1005000069642063686F69636573206172653A206E
:100510005B315D2D5B31365D20286368616E6E65F1
:100520006C20312D31362900536574206F7574703D
:10053000757420666F7220706F727420005B585D56
:100540002061626F7274206368616E6765732061F9
:100550006E64206578697420525820636F6E6669F6
:1005600067005B535D207361766520736574746901
:100570006E677320746F205258005B525D20726565
:10058000766572742052582073657474696E67734F
:1005900020746F2064656661756C747300557365B3
:1005A000206E756D62657273205B312D445D207421
:1005B0006F206564697420706F727473205B452DC1
:1005C000515D20666F722073657474696E67730085
:1005D000202D20726563656976657220636F6E6693
:1005E0006967757261746F722C207278207377203E
:1005F000000A0A6F70656E4C52536E672000536597
:10060000742073657269616C2062617564726174D3
:10061000653A200056616C69642063686F696365A0
:10062000733A2031202D20342B34202F2032202DDE
:100630002038202F2033202D20382B34202F203419
:10064000202D203132202F2035202D2031322B3407
:10065000202F2036202D203136005365742043682A
:10066000616E6E656C20636F6E6669673A20005339
:1006700065742044617461726174652028302D3284
:10068000293A200053657420486F70206368616EBA
:100690006E656C7320286D61782032342C20736570
:1006A0007061726174656420627920636F6D6D6141
:1006B00073292076616C69642076616C756573209E
:1006C000312D3235353A2000536574206368616EF0
:1006D0006E656C2073706163696E672028783130B5
:1006E0006B487A293A200053657420524620706F77
:1006F0007765722028302D37293A20005365742001
:100700005246206D616769632028686578292065F5
:100710002E672E20307844454144463030443A20FC
:10072000005365742062617365206672657175653A
:100730006E63792028696E20487A293A20005B5A36
:100740005D20656E74657220726563656976657299
:1007500020636F6E66696775726174696F6E20756C
:1007600074696C79005B465D20646973706C6179B3
:100770002061637475616C206672657175656E6366
:100780006965732075736564005B525D2063616CFD
:1007900063756C6174652072616E646F6D206B654A
:1007A0007920616E6420686F70206C697374005BDF
:1007B000495D207265696E697469616C697A65204A
:1007C00073657474696E677320746F20736B6574DE
:1007D00063682064656661756C7473005B585D20A6
:1007E000726576657274206368616E6765732061F7
:1007F0006E642065786974206D656E75005B535D6D
:1008000020736176652073657474696E67732074F4
:100810006F20454550524F4D20616E6420657869C8
:1008200074206D656E7500557365206E756D62651B
:100830007273205B302D395D20746F20656469749C
:1008400020706172616D657465727300202D205394
:10085000797374656D20636F6E6669677572617414
:10086000696F6E000A0A6F70656E4C52536E672096
:10087000005129204F7574707574206265666F721F
:1008800065206C696E6B20283D465329203A200074
:10089000502920536C617665206D6F646520286552
:1008A00078706572696D656E74616C293A20004FCD
:1008B000292054696D65642042494E4420617420AA
:1008C0007374617274757020203A20004E29205094
:1008D000504D206F7574707574206C696D69746506
:1008E0006420202020203A200044495341424C45B6
:1008F00044004D292050504D205253534920746FCD
:10090000206368616E6E656C202020203A20004CC8
:10091000292050504D206D696E696D756D20737979
:100920006E63202875732920203A200044495341E2
:10093000424C4544004B29204661696C73616665F1
:1009400020626561636F6E20696E74762E20283197
:100950002D32353573293A20004A29204661696CC9
:100960007361666520626561636F6E2064656C61AA
:10097000792028302D323535203D3E20313073200E
:100980002D203135306D696E293A200049292046E5
:1009900061696C7361666520626561636F6E206674
:1009A00072712E203A200048292050574D20737430
:1009B0006F702064656C6179202020202020203A0F
:1009C000200047292050504D2073746F70206465BB
:1009D0006C6179202020202020203A200046292008
:1009E0004661696C736166652064656C617920207D
:1009F00020202020203A200050574D206368616E4F
:100A00006E656C200066756E6374696F6E3A2000C7
:100A10002920706F72742000506F776572546F7761
:100A2000657200445446205548462033322D626991
:100A3000742031306368004F70656E4C52536E679E
:100A40005258206D696E6920342F36636800466CF9
:100A50007974726F6E2F4F72616E676552582055B0
:100A600048462038636800525820747970653A20EF
:100A70000044697361626C656400487A00203D3D02
:100A8000200043616C63756C617465642070616300
:100A90006B657420696E74657276616C3A200042F1
:100AA00029204D6963726F202868616C6629205087
:100AB000504D202020203A00412920496E76657251
:100AC0007465642050504D20696E20202020203A0B
:100AD000003029204D7574652062757A7A65722020
:100AE000286D6F73746C79293A0039292053657227
:100AF00069616C2062617564726174653A00736D3E
:100B0000617274506F7274004672536B7900547244
:100B1000616E73706172656E740044697361626CBA
:100B200065640038292054656C656D657472793A86
:100B300020202020202020003729204368616E6E6D
:100B4000656C20636F6E6669673A20200036292045
:100B500044617461726174652028302D32293A2015
:100B6000202000352920486F70206368616E6E6513
:100B70006C733A2020202020003429204368616EC5
:100B80006E656C2073706163696E673A2020003374
:100B90002920524620706F7765722028302D372922
:100BA0003A202020003229205246206D6167696377
:100BB0003A202020202020202020003129204261BE
:100BC0007365206672657175656E63793A202020C1
:100BD0000000000000240027002A0000000000257B
:100BE0000028002B0000000000230026002900043C
:100BF00004040404040404020202020202030303C4
:100C000003030301020408102040800102040810BD
:100C1000200102040810200000000700020100006B
:100C2000030406000000000000000000F52E11245F
:100C30001FBECFEFD8E0DEBFCDBF13E0A0E0B1E034
:100C4000ECE2F0E602C005900D92A839B107D9F7A1
:100C500016E0A8E9B3E001C01D92A935B107E1F79C
:100C60001CE0CEE2DCE004C02297FE010E94F12FDE
:100C7000CC32D107C9F70E943A2F0C9414300C944F
:100C80000000A0E0B0E0E7E4F6E00C94C02FEC0137
:100C9000A880B980CA80DB80A114B104C104D1044A
:100CA00041F484E2A82E89EDB82E8BE5C82E87E0AA
:100CB000D82EC601B5012DE133EF41E050E00E948E
:100CC0009D2F27EA31E440E050E00E94492F7B014C
:100CD0008C01C601B5012DE133EF41E050E00E94E7
:100CE0009D2FCA01B9012CEE34EF4FEF5FEF0E9448
:100CF000492F6E0D7F1D801F911F97FF04C061500B
:100D0000704080409048688379838A839B839B01ED
:100D1000AC015F77B901CA01CDB7DEB7EAE00C9448
:100D2000DC2F0E944106089581EB92E00E9441066B
:100D300008956093B1027093B2028093B3029093CE
:100D4000B4020895A0E0B0E0E8EAF6E00C94B92F10
:100D5000EC012B016A016115710519F0FB0191830A
:100D60008083C114D10449F0C6010297839728F00B
:100D700020E030E040E050E0DCC0A9908A2D90E017
:100D80000E940930892BC9F7FDE2AF1621F4A99022
:100D90003324339405C08BE2A81609F4A9903324B8
:100DA000C114D10421F0E0E1CE16D10411F5F0E335
:100DB000AF1669F48881883711F0883541F4A9802D
:100DC000229682E0382A20E1C22ED12C12C0C11412
:100DD000D10479F4E0E3AE1659F199E9E92E99E9E5
:100DE000F92E99E9092F99E1192F8AE0C82ED12C03
:100DF0003AC0FAE0CF16D10491F080E1C816D104D0
:100E000029F0E8E0CE16D104F9F415C0BFEFEB2EBF
:100E1000BFEFFB2EBFEF0B2FBFE01B2F24C0A9E9B4
:100E2000EA2EA9E9FA2EA9E90A2FA9E11A2F1BC077
:100E3000F8E0CF2ED12CEFEFEE2EEFEFFE2EEFEFFE
:100E40000E2FEFE11E2F0FC09601442737FD40956E
:100E5000542F6FEF7FEF8FEF9FEF0E947B2FC90121
:100E6000DA017C018D0120E030E040E050E060E0FC
:100E70003601882477FC8094982C70EDB72EBA0C3C
:100E8000F9E0FB1570F48A2D81548A3118F499EC3D
:100E9000B92E06C08A2D81568A3148F589EAB82EC6
:100EA000BA0C8B2D90E08C159D050CF56F3FE9F089
:100EB000E216F30604071507B8F0CA01B901A40148
:100EC00093010E94492F9B01AC018B2D90E0A0E083
:100ED000B0E0280F391F4A1F5B1F281739074A0740
:100EE0005B0710F061E001C06FEFA990C6CF41141D
:100EF000510451F0662311F0219703C031FE04C064
:100F00002297F201D183C08330FE07C050954095EF
:100F1000309521953F4F4F4F5F4F67FF0AC082E2E8
:100F200090E090935806809357062FEF3FEF4FEFD6
:100F30005FEFB901CA01CDB7DEB7E1E10C94D52F5F
:100F4000FC0188279927E89421912032E9F3293080
:100F500010F02E30C8F32B3241F02D3239F4689462
:100F600004C00E94F507820F911D219120532A3061
:100F7000C0F31EF4909581959F4F089548E953E082
:100F80000E94C3070895009731F4DA018D919C9176
:100F9000009709F40EC0DC01FB013D912191222351
:100FA00019F03217C9F3FACF332331F4DA011D9265
:100FB0001C928827992708951197AF93BF93FB013F
:100FC0003D912191321771F4332321F48827992719
:100FD000119702C01E921196FA01A193B0839F91BE
:100FE0008F910895222369F7EACF7AE0979F902D99
:100FF000879F802D910D1124089580919A0381304F
:1010000019F482E080939A0380919A03833019F453
:1010100084E080939A030895E3E0F0E089E0809310
:101020005700849190E08670863009F491E0892F12
:1010300008951F93182F0E940C08882379F09FB7FA
:1010400081E080939F05F894A89588E180936000E3
:1010500010936000112309F0A8959FBF1F91089578
:10106000382F20E080913105909132058227932717
:1010700040E061E270E19C01220F331F97FF04C042
:10108000C9018627972701C0C9014F5F483099F7EA
:101090009093320580933105089587E38093D003C0
:1010A00080E092ECA1E0B0E08093D1039093D20372
:1010B000A093D303B093D40387E08093DD0380EC47
:1010C0009AECA9E8B6E38093D5039093D603A09356
:1010D000D703B093D80385E08093DE038DEE9EEFB7
:1010E000ADEABEED8093D9039093DA03A093DB03BE
:1010F000B093DC03AFEDB3E080E090E0863010F019
:10110000E0E004C0FC01EF57FC4FE081ED93019655
:101110008831910599F782E08093F7038AE0809304
:10112000F803089580EC97EFAAEBB7E380939D0353
:1011300090939E03A0939F03B093A00380E090E060
:10114000A0E0B0E58093A1039093A203A093A30332
:10115000B093A403E5EAF3E080E081938F5F8031F0
:10116000E1F708958436910520F4BC0180E090E019
:1011700025C08E3B910550F48A559040BC0180E01B
:1011800090E02AE030E040E050E016C0823D91055A
:1011900050F4845B9040BC0180E090E024E630E0B5
:1011A00040E050E009C08D5C9040BC0180E090E0E0
:1011B00028E532E040E050E00E94492F24E630E08C
:1011C00040E050E00E94492F089590E08C599F4FD5
:1011D0000E94B2080895DC019896EC91F0E0E77067
:1011E000F070E758FC4F808108958F929F92AF92E4
:1011F000BF92CF92DF92EF92FF920F931F938C01D9
:101200000E94EB08D80197962C9130E043E150E022
:10121000249FF001259FF00D349FF00D1124EB5415
:10122000FD4F80809180A280B38090E00F96AA2726
:1012300097FDA095BA2FBC01CD0120E43FE14DE719
:1012400050E00E94492FA50194010E947B2F690163
:101250007A0180ED97E0A0E0B0E0C80ED91EEA1E4A
:10126000FB1ED80198968C91887181F060E07EEE2B
:101270008AEB9BE0A50194010E947B2F28513C4FF3
:101280004F4F5F4FC20ED31EE41EF51E87EE93E054
:10129000A0E0B0E0C80ED91EEA1EFB1EC701B601D1
:1012A00028EE33E040E050E00E947B2FCA01B901F4
:1012B00028EE33E040E050E00E94492F1F910F914B
:1012C000FF90EF90DF90CF90BF90AF909F908F9066
:1012D00008958F3F910509F010F480E0089522E011
:1012E0008030920710F481E008958050934010F010
:1012F00083E0089582E00895CF92DF92FF920F93EA
:101300001F93CF93DF93F82FEB016A01182F1695E7
:10131000E0E088819981D6018C938A819B81119626
:101320008C9311978C819D8112968C9312978E814C
:101330009F8113968C931397288139814A815B8111
:101340006C817D818E819F819295990F990F907C00
:10135000832F8370982B852F8370880F880F982B8D
:10136000872F83708295807F982B14969C9385E0BD
:1013700090E0C80ED91E2896EF5F1E1750F6F0FFBA
:1013800021C0888199810E946909F82E8A819B81F8
:101390000E946909182F8C819D810E946909082F7C
:1013A0008E819F810E946909F294FF0CFF0C70EC02
:1013B000F7221295107F1F29182B000F000F012B09
:1013C000D6010C93DF91CF911F910F91FF90DF9089
:1013D000CF90089523E08032920718F420E030E0A7
:1013E00026C023E0883E920748F49C012F513340E9
:1013F00054E0369527955A95E1F719C027E0803DCE
:10140000920720F49C012C5D334011C028E08839FC
:10141000920718F02FEF33E00AC09C01285C374098
:1014200044E0369527954A95E1F72D503C4FC90188
:1014300008958C30910548F49C0174E0220F331F0D
:101440007A95E1F7285D3C4F17C023E0843F92076F
:1014500020F49C0124523C4F0FC024E080309207BE
:1014600018F020E938E008C09C012657334F64E0AB
:10147000220F331F6A95E1F7C90108959C01369543
:10148000279525753575821B930B9C0136952795FD
:10149000369527952373337383739373280F391FFE
:1014A000C901E4E096958795EA95E1F7820F931FCD
:1014B0008F709F7021E031E0AC01429FC001439FDB
:1014C000900D529F900D1124892F0895882339F093
:1014D0005F980000289A00005F9A000008955F98C6
:1014E0000000289800005F9A000008955F9A0000AD
:1014F00083B15F98000090E096958795817008957C
:101500000F931F93082F5C9A5F985C9810E0802FD0
:1015100080780E94660A000F1F5F1830C1F75F983D
:101520001F910F9108958F770E94800A08950F935D
:101530001F93082F10E0802F80780E94660A000F0A
:101540001F5F1830C1F75F981F910F9108950F9397
:101550001F935F9880E000E0182F110F0E94760A19
:10156000810F0F5F0830C1F71F910F9108950E94FE
:10157000930A0E94A70A5C9A08951F93162F806809
:101580000E94800A812F0E94970A5C9A1F910895F9
:101590001F931091D9031827E0EDF3E0E80FF11D38
:1015A00089E767850E94BD0A8DE3612F0E94BD0A0D
:1015B00082E4612F0E94BD0A1F91089586E20E9475
:1015C000B70A08950F931F938C018CE1F801648191
:1015D0000E94BD0A8DE1F80165810E94BD0A8EE17D
:1015E000F80166810E94BD0A80E2F80167810E94CD
:1015F000BD0A81E2F80160850E94BD0A82E2F8011D
:1016000061850E94BD0A83E2F80162850E94BD0ADD
:1016100084E2F80163850E94BD0A85E2F8016485D1
:101620000E94BD0A8AE2F80165850E94BD0A8EE625
:10163000F80166850E94BD0A8FE6F80167850E9461
:10164000BD0A80E7F80160890E94BD0A81E7F801C0
:1016500061890E94BD0A82E7F80162890E94BD0A81
:101660001F910F910895EF92FF920F931F93CF93C5
:10167000DF937B018C01603028E372072CE982073D
:101680002CE1920728F520E836E948E950E00E946D
:101690007B2FE9016897B90180E090E020E839E606
:1016A00047E65FEF0E94492F6E0D7F1D801F911F3F
:1016B00032E0660F771F881F991F3A95D1F721E70F
:1016C00032E040E050E00E947B2F890180E421C09D
:1016D00020E03DE241E351E00E947B2FE901689761
:1016E000B90180E090E020E033ED4EEC5EEF0E9427
:1016F000492F6E0D7F1D801F911F660F771F881F5A
:10170000991F21E732E040E050E00E947B2F8901E1
:1017100080E69E012F71622F680F85E70E94BD0A47
:1017200086E7612F0E94BD0A87E7602F0E94BD0AED
:10173000CDB7DEB7E6E00C94E02F9F92AF92BF9258
:10174000CF92DF920F93DF93CF9300D000D0CDB72D
:10175000DEB7982E83E00E94B70A8093F90384E0F5
:101760000E94B70A8093FA0386E060E00E94BD0AF7
:1017700087E061E00E94BD0A89E06FE70E94BD0A30
:101780008AE065E00E94BD0A8BE062E10E94BD0A2A
:101790008CE065E10E94BD0A8DE06DEF0E94BD0AFC
:1017A0008EE060E00E94BD0A992019F084E193E088
:1017B00008C08091F70323E1829FC00111248B545C
:1017C0009D4F0E94E20A80E36CE80E94BD0A82E31A
:1017D0006FE00E94BD0A83E362E40E94BD0A84E3D5
:1017E0006AE00E94BD0A85E36AE20E94BD0A86E3C0
:1017F0006DE20E94BD0A87E364ED0E94BD0A88E3A2
:1018000060E00E94BD0A89E360E00E94BD0A992061
:1018100049F065E8A62E61ECB62E61ECC62E6EEDA1
:10182000D62E08C0A090D903B090DA03C090DB0395
:10183000D090DC030AE38D2D9927AA27BB27898343
:101840009A83AB83BC83802F69810E94BD0A802F5D
:101850008B5F69810E94BD0ADC2CCB2CBA2CAA2498
:101860000F5F0E3341F783E46FEF0E94BD0A84E4FB
:101870006FEF0E94BD0A85E46FEF0E94BD0A86E407
:101880006FEF0E94BD0A992019F08DE666E003C053
:101890008DE66091DD030E94BD0A89E760E00E9449
:1018A000BD0A8AE76091DE030E94BD0A83E760E01B
:1018B0000E94BD0A84E760E00E94BD0A992029F0D9
:1018C00060EC7AEC89E896E308C06091D5037091EA
:1018D000D6038091D7039091D8030E94330B0F90C9
:1018E0000F900F900F90CF91DF910F91DF90CF90DD
:1018F000BF90AF909F90089587E061E00E94BD0A7D
:101900008EE764E20E94BD0A88E063E00E94BD0A9F
:1019100088E060E00E94BD0A87E065E00E94BD0AA1
:1019200085E062E00E94BD0A83E00E94B70A8093CE
:10193000F90384E00E94B70A8093FA030895582FB0
:1019400040919E04842F90E0FC01EF70F0709F01A5
:101950002F5F3F4F74E0959587957A95E1F72817AB
:10196000390751F0E257FB4F5083842F8F5F8F7000
:10197000407F842B80939E0408951F920F920FB690
:101980000F921124EF92FF920F931F932F933F9387
:101990004F935F936F937F938F939F93AF93BF9377
:1019A000EF93FF93E090A103F090A2030091A303B3
:1019B0001091A40389B1A801970120743070407080
:1019C000507090E063E0969587956A95E1F7A0E006
:1019D000B0E081709070A070B070281739074A0786
:1019E0005B0709F46AC02091840030918500109251
:1019F0008500109284008091BF04882309F05DC0A7
:101A0000E5FC02C03695279589E0253C3807C8F1EA
:101A100080914703A80197011CE15695479537959A
:101A200027951A95D1F7211531054105510521F466
:101A300021E030E040E050E090E0A0E0B0E0281786
:101A400039074A075B07D0F4809147038F3FB1F015
:101A500020E00EC0E22FF0E0EE0FFF1FDF01A054E8
:101A6000BB4F8D919C91E95DFC4F918380832F5FEB
:101A700080914703281770F31092BE041092470319
:101A80001CC082E02D3B3807A8F0809147038031CD
:101A900088F410914703C9010E94EA09E12FF0E0A0
:101AA000EE0FFF1FE054FB4F918380831F5F109365
:101AB000470303C08FEF80934703FF91EF91BF91DE
:101AC000AF919F918F917F916F915F914F913F91D6
:101AD0002F911F910F91FF90EF900F900FBE0F90DD
:101AE0001F90189583E0809380008AE180938100A5
:101AF0008FEF9FEF909389008093880010926F0082
:101B000088E080936D00E8E6F0E080818460808367
:101B100008956F3018F086958058089589E0689F81
:101B2000802D11240895882319F460E071E002C02B
:101B300063E071E085E396E00E94FD2C0895A0E04B
:101B4000B0E0E5EAFDE00C94C22F182F0E94AE2908
:101B50009B01AC0180912B0590912C05A0912D0546
:101B6000B0912E0569017A01C81AD90AEA0AFB0A5E
:101B7000D701C60189589341A040B04010F010929F
:101B80002A0520932B0530932C0540932D05509367
:101B90002E052091BF04822F81508230E8F580917C
:101BA0002A05882309F44FC1813011F482E0BCC1B9
:101BB000803108F035C1E82FF0E0E054FB4F10838E
:101BC0008F5F80932A05803109F0B0C1A2ECB4E0A8
:101BD000213039F41196EC911197E695E6958C91A8
:101BE00009C08D919C911197E92FE695E695E695B0
:101BF00096958795E03140F4F0E090E0EE0FFF1FFE
:101C0000E95DFC4F918380831092BE04129684E0BC
:101C1000A03DB807E9F68AC1233009F004C18091DC
:101C20002A05882321F41F3009F080C10CC18831B6
:101C300030F4E82FF0E0E154FB4F108374C1883199
:101C400009F0EEC0112309F0EBC0C0E0D0E00BE0DA
:101C500010E0DE0163E0AA0FBB1F6A95E1F7C09FA9
:101C6000B001C19F700DD09F700D1124FB01E05495
:101C7000FB4F80812181922F977095958795FD016B
:101C8000EE0FFF1FE95DFC4F91838083FB01EF5353
:101C9000FB4F30813695369536952181422F4295FE
:101CA000440F407E842F832B269526952695922FD0
:101CB000977095958795FD01EE0FFF1FE75DFC4F2F
:101CC00091838083FB01EE53FB4F80818295869543
:101CD000869583704181942F990F990F292F282B76
:101CE000429546954695437082818170880F880F92
:101CF000382F342B35952795FD01EE0FFF1FE55D3D
:101D0000FC4F31832083FB01EC53FB4F3081369530
:101D10002181422F479544274795842F832B269571
:101D2000922F977095958795FD01EE0FFF1FE35D4C
:101D3000FC4F91838083FB01EB53FB4F3081329545
:101D40003F702181422F4295407F842F832B229523
:101D50002F70922F977095958795FD01EE0FFF1FBD
:101D6000E15DFC4F91838083FB01EA53FB4F80814F
:101D7000881F8827881F4181942F990F292F282B8E
:101D8000441F4427441F82818370880F382F342BCF
:101D900035952795FD01EE0FFF1FEF5CFC4F31835A
:101DA0002083FB01E853FB4F308136953695218126
:101DB000422F4295440F440F407C842F832B26955D
:101DC0002695922F977095958795AA0FBB1FFD01B9
:101DD000ED5CFC4F9183808367537B4FFB01208137
:101DE0002295269527704181342F330F330F330FFF
:101DF000832F822B942F9295969597709595879522
:101E0000AB5CBC4F11969C938E932196C230D1054A
:101E100009F01FCF8091D60483FD02C01092BE044A
:101E200010922A0583C0243009F080C040912A0511
:101E3000442359F4183AB1F4109232051092310546
:101E400088EA0E94300881E06FC0413019F4109395
:101E50002F0504C0423031F410933005812F0E94C9
:101E600030085DC060913005262F30E0220F331F0F
:101E7000E42FF0E0C90102968E179F0734F0433239
:101E800068F7E354FB4F1083E9CF2D5F3F4F40913C
:101E9000310550913205E217F30749F4912F80E0A4
:101EA00048275927509332054093310538C0812F78
:101EB00090E04817590789F580912F05813069F521
:101EC000613118F080E180933005D0903005F0EC5E
:101ED000EF2EF4E0FF2E00E010E01BC0F701D081F0
:101EE000C0E0818190E08C2B9D2BE3E09695879557
:101EF000EA95E1F70E94EA09F801EE0FFF1FE95D9C
:101F0000FC4F918380830F5F1F4F82E090E0E80ECB
:101F1000F91E0D1518F31092BE0410922A05809137
:101F20002A05882319F08F5F80932A05CDB7DEB785
:101F3000E8E00C94DE2FFF920F931F93CF93DF9373
:101F4000182F092FF62E8EE30E94BD0A212F302F65
:101F5000C901EC0110E005C08FE769910E94BD0A3C
:101F60001F5F1F15C8F385E064E00E94BD0A83E08F
:101F70000E94B70A8093F90384E00E94B70A809315
:101F8000FA030E94AE296093FB037093FC038093D5
:101F9000FD039093FE0387E069E00E94BD0A81E0A3
:101FA00080939A03CDB7DEB7E5E00C94E12F0E9451
:101FB0009B0F80919A038130D9F40E94AE29209121
:101FC000FB033091FC034091FD035091FE03621B23
:101FD000730B840B950B605A76488140904040F417
:101FE000E8CF85E396E067E071E00E94FD2C08955C
:101FF00080919A038130A9F3089585E396E06EE716
:102000000E94B52E0895A0E0B0E0E9E0F0E10C9464
:10201000C12F6C0185E396E06EE70E94B52E760134
:1020200000E010E0C0E0D0E0B0E2BB2E0AC0083013
:10203000110521F49E012095F60120870894E11CEA
:10204000F11CF7016081862F8D57823040F485E3C3
:1020500096E06DE70E94B52EF70160816B2585E360
:1020600096E00E94B52E0115110551F0F70180810F
:102070009E01280F311DC32FDD27C20FD31FD07043
:102080000F5F1F4F0930110591F6CDB7DEB7E9E0BC
:102090000C94DD2FA9E0B0E0E0E5F0E10C94C82F4E
:1020A000382FE62F8091A30490E0019664E270E05F
:1020B0000E94682F982F8093A30488E9898380E188
:1020C0008A83913071F0913028F0923099F09330FA
:1020D000E1F416C085E08B8381EF8C832F5F2D8325
:1020E00017C09B8381EF8C8384E6489FC001112435
:1020F0009D830EC084E08B8381EF8C833D8308C079
:102100009B8381EF8C83ED8303C00E94FD0F04C08D
:10211000CE0101960E9403102996E2E00C94E42F70
:102120000F931F93CF93DF93182F092F85E396E02A
:102130006EE70E94B52E212F302FC901EC0110E06F
:1021400000E288818D57823040F485E396E06DE7A8
:102150000E94B52E88818027888385E396E0699167
:102160000E94B52E1F5F193061F785E396E06EE798
:102170000E94B52EDF91CF911F910F910895A9E094
:10218000B0E0E5ECF0E10C94C82F382F8091A30467
:10219000882379F48EEF89833A836B83842F90E0D0
:1021A000959587958C832D83198618861F821E82AC
:1021B0002FC040919E04842F90E09C012F703070BE
:1021C00054E0959587955A95E1F78217930721F189
:1021D0008DEF89831A821B82DE01149620E008C0ED
:1021E000E257FB4F80818D93405F2F5F263069F06F
:1021F000842F90E0FC0134E0F595E7953A95E1F7FE
:102200008F709070E817F90759F740939E042A835E
:10221000CE0101960E9490108091A30490E0019657
:1022200066E070E00E94682F8093A3042996E2E0A4
:102230000C94E42F9F92AF92BF92CF92DF92EF92D5
:10224000FF920F931F93B82EA62ED42EC22E902E3F
:102250000E94AE297B018C0180918D0420919F0406
:102260003091A0044091A1045091A2048823B1F0C0
:10227000D801C701821B930BA40BB50B815E9E4254
:10228000A040B04020F12C2DDC1408F42D2D8B2D16
:102290006A2D422F292D0E944A1011C0D801C70172
:1022A000821B930BA40BB50B81539547A040B04004
:1022B00070F08B2D6A2D4D2D2C2D0E94BF10E092B9
:1022C0009F04F092A0040093A1041093A2041F9114
:1022D0000F91FF90EF90DF90CF90BF90AF909F90C5
:1022E000089585E396E0609100040E94B52E08955C
:1022F0001F93182F85E396E0612F0E94B52E8091E1
:1023000000048127809300041F9108951F93192FC3
:102310000E947811812F0E9478111F910895DF92F9
:10232000EF92FF920F931F93D82E7B01109200041F
:1023300005E316E0C80165EB0E94B52EC80162E610
:102340000E94B52E8D2D0E947811C7010E94861122
:102350001F910F91FF90EF90DF900895E82FF0E02C
:10236000E456FC4FE185E03158F4F894F0E0EE0FCC
:10237000FF1FE95DFC4F0190F081E02D78940DC0C6
:10238000E03129F0E13129F0E0E0F2E006C082E13D
:1023900001C083E10E94022BFC01CF01089589E076
:1023A00060E00E94332A88E061E00E94332A87E0DF
:1023B00061E00E94332A82E060E00E94332A84E0D8
:1023C00061E00E94332A0895892B19F08AE061E0C8
:1023D00002C08AE060E00E949F2A0895A0E2B0E077
:1023E000E4EFF1E10C94C02F8CE00E94B70A88233F
:1023F00079F585E396E063E171E00E94FD2C2D9A6A
:1024000080E00E949D0B0E947C0C2D9821C085E3EA
:1024100096E00E947C2E482F8091BF04882321F0F3
:10242000842F0E949F0D14C080912805E82FF0E0B2
:1024300031969F012F71307031978091270590E080
:102440002817390729F0E250FB4F408320932805D5
:1024500085E396E00E94422E892BC9F680919A036B
:10246000843009F08EC00E94AE296093AE04709350
:10247000AF048093B0049093B10461157105810598
:10248000910561F481E090E0A0E0B0E08093AE04BB
:102490009093AF04A093B004B093B1048091BA04B8
:1024A0009091BB0481609093BB048093BA0483E055
:1024B00080939A038FE70E94930A05EF14E00E942D
:1024C000A70AF80181938F01F4E00E3F1F07B9F7C7
:1024D0004091E0048091F504282F30E0842F90E0B3
:1024E0008227932786FF40C080E448274093E0047A
:1024F000C90188739070C89709F510E014C01F5F78
:102500008091F803E12FF0E084FF06C0EB50FB4F11
:1025100080810E949F0C07C0EB50FB4F85E396E043
:1025200060810E94B52E212F30E08091F50490E06B
:10253000877090708217930714F716C02F7330704E
:10254000232B91F48091F6048093B2048091F704D8
:102550008093B4048091F8048093B5048091FB04C7
:102560008093BC041092BD0480912905813019F438
:1025700082E08093290580912905833011F410921F
:1025800029050E94AE295B016C018091B6049091EF
:10259000B704A091B804B091B9040097A105B105A2
:1025A000C9F086017501E81AF90A0A0B1B0BD8015C
:1025B000C701885B9B40A040B04060F00E94DE0AEB
:1025C0008093B3041092B6041092B7041092B8042A
:1025D0001092B90480ED93E00E94F5082091AA04BE
:1025E0003091AB044091AC045091AD04860175016B
:1025F000E21AF30A040B150BE616F706080719078B
:1026000008F40CC1A092AA04B092AB04C092AC042E
:10261000D092AD04A8958091BE048830A0F080913E
:10262000A1039091A203A091A303B091A403FCE1A4
:10263000B695A79597958795FA95D1F70097A10537
:10264000B10509F08AC18091BE048F5F8093BE04FA
:10265000E090AE04F090AF040091B0041091B1048A
:10266000E114F1040105110511F180ED93E00E94E0
:10267000F508AE18BF08C00AD10A6A157B058C059B
:102680009D0588F48091A10384FD04C080ED97E04E
:102690000E94E4111092AE041092AF041092B004A4
:1026A0001092B10404C080E090E00E94E411909187
:1026B000E004907C9093E004009128051091270598
:1026C0000117B1F180912905823091F590589093CE
:1026D000E00480ED93E00E94EB08893010F048E0C0
:1026E00002C0482F415030E013C03F5FA32FB0E03D
:1026F000812F90E0FC01E250FB4F2081FD01E05270
:10270000FB4F2083A25EBA4F2C930196182F1F71A6
:10271000341710F4101749F710932705832F895C9D
:102720009091E004892B8093E00430931E051AC039
:10273000209129052430D1F490911E05EFE1F5E0B8
:10274000A1EEB4E0292F30E02E0F3F1F02C081918F
:102750008D93E217F307D9F7995C8091E004982BE9
:102760009093E00483E08093290536C08091A5040E
:10277000823059F491609093E0042D9A05EA13E0B9
:102780007E010894E11CF11C10C09093E0042D9888
:10279000222319F481E08093290580912905833053
:1027A00069F784E080932905E9CFF80181918F01D1
:1027B0000E94AE11F701819391937F01F3E0053BF5
:1027C0001F0799F78091F8038770BE016F5F7F4FF5
:1027D00041EE54E00E947C092C9A8091A4040E944E
:1027E000C80A80ED93E00E94EB08682F80EE94E029
:1027F0000E949B0FE091A404EF5FE093A404E831F2
:1028000031F0F0E0E053FC4F8785882339F41092D3
:10281000A40404C02D9A89E08093BE048091F8033B
:10282000887171F180919A03823051F58091BA04D8
:102830009091BB04880F991F9093BB048093BA04B6
:1028400083E080939A030E947C0C0E94AE296093DF
:10285000B6047093B7048093B8049093B9046115DB
:1028600071058105910561F481E090E0A0E0B0E0A0
:102870008093B6049093B704A093B804B093B904BE
:102880008091F80384FF1EC08091BA049091BB042C
:102890008E7F0E943E0A182F8091B2046091BC0482
:1028A0000E94890D082F8091B304612F0E94890D29
:1028B000282F8091B4046091B504402F00919B03B0
:1028C0000E941A112C988091A5048130D1F081309A
:1028D00020F0823009F047C034C08BE00E94D22A39
:1028E000892B09F040C081E08093A5040E94A029B3
:1028F0006093A6047093A7048093A8049093A904FE
:1029000032C08BE00E94D22A892B21F50E94A02997
:102910002091A6043091A7044091A8045091A904E5
:10292000621B730B840B950B695E73408040904073
:10293000D0F082E08093A50480ED97E00E94E4113E
:1029400012C08BE00E94D22A892B69F080E090E0CF
:102950000E94E4111092A50406C08091BE04883044
:1029600009F059CF57CFA096EAE00C94DC2F8AE00B
:1029700061E00E94332A8AE060E00E949F2A089565
:102980001F93182F0E94AE2960939F047093A00498
:102990008093A1049093A20410938D04112329F431
:1029A00040E855E260E070E004C040E051EE60E0D5
:1029B00070E085E396E00E94BB2D1F910895ACE185
:1029C000B0E0E5EEF4E10C94C02F0E94AE297B014B
:1029D0008C0181E00E949D0B84E7A82E6E01089473
:1029E000C11CD11CB3E0BB2EA982C60161E00E94CC
:1029F000D70FB0929A030E947C0C6AEF70E080E0DF
:102A000090E00E94D42980919A03833009F07DC020
:102A100085E396E00E94422E892B09F076C00E9441
:102A2000AE296E197F09800B910B6058734C894C4D
:102A3000914008F06AC0D8CF8FE70E94930A0E94A5
:102A4000A70A843509F05CC089830E94A70A182F61
:102A500000E010938C0400938B040E94A70A080FD7
:102A6000111D10938C0400938B040E94A70A80937D
:102A70008A040E94A70A80938904813108F040C02B
:102A8000FF2407C00E94A70A07591B4FF801808343
:102A9000F3940F2D10E08091890490E0880F991F26
:102AA0000817190778F380E78983CE01019661E062
:102AB0000E94D70F83E080939A030E947C0C62E30C
:102AC00070E080E090E00E94D42980919A038330E6
:102AD000A9F08FE70E94930A0E94A70A803581F42B
:102AE000898305EB13E00E94A70AF80181938F0107
:102AF000F3E0003D1F07B9F781E003C082E001C0A9
:102B000083E06C96EAE00C94DC2F80919A0383308A
:102B100009F092CFF3CF83E00E94B70A8093F903C4
:102B200084E00E94B70A8093FA0387E061E00E9484
:102B3000BD0A6AE070E080E090E00E94D4290E9423
:102B40007C0C000008950F931F93082F17C02D9A37
:102B500064E670E080E090E00E94D4292D9864E65D
:102B600070E080E090E00E94D4291F5F101778F396
:102B70006CE271E080E090E00E94D42910E0F6CF92
:102B8000482F392F25E00DC0F999FECF1FBA842FA9
:102B9000932F92BD81BD60BD0FB6F894FA9AF99A51
:102BA0000FBE215059F0F999FECF842F932F92BD7B
:102BB00081BDF89A80B5681739F7089582E00E94C0
:102BC000A3150895A0E0B0E0E8EEF5E10C94B92F6C
:102BD000482E562ECC24DD24EE24FF24882499246C
:102BE000C0E0D0E076E4372E04C0CC24DD245524A8
:102BF0005394442069F480919B03839DE001112448
:102C00006CE9E62E63E0F62E59E1852E912C1DC06D
:102C100021E0421671F480919B03839DE001112411
:102C20006B9640EDE42E43E0F42E39E2832E912C96
:102C30000CC032E0431649F42BE9E22E23E0F22ED9
:102C400091E0892E912CC8E1D1E03E016C0C7D1CF5
:102C50001092320510923105E3011BC0552059F442
:102C6000F999FECFD2BDC1BDF89A80B5F701E00F4A
:102C7000F11F808307C0F701E00FF11FCE016081D3
:102C80000E94C0150E0D1F1DF80180810E943008A2
:102C900021969E012619022F10E008151905F0F261
:102CA000CE015520D9F4F999FECFD2BDC1BDF89A15
:102CB00020B5F999FECF2196D2BDC1BD2197F89AD2
:102CC00080B590E0B22EAA248A299B292091310553
:102CD000309132052817390759F487CF2196609132
:102CE00032050E94C015CE01609131050E94C015C9
:102CF00080E291E0C80ED91E91EEC91692E0D90685
:102D000008F477CF852DCDB7DEB7E1E10C94D52F50
:102D100080E061E00E94E21581E061E00E94E2153E
:102D2000089580E060E00E94E215882331F081E0A0
:102D300060E00E94E215882331F40E9492080E940C
:102D40004D080E948816089582E061E00E94E21515
:102D5000089582E060E00E94E21580919B03843038
:102D600020F010929B030E94A41608951F93182F21
:102D70000E94A91680919B03811731F0143020F432
:102D800010939B030E94A4161F910895109267044C
:102D900085E6E2E0F4E0DF011D928A95E9F7089507
:102DA0001F93182F8F3711F08830E1F5E0916704F9
:102DB000EE2309F455C0E150E0936704F0E0EE5FC4
:102DC000FB4F108285E396E06DE00E94B52E10E087
:102DD0000AC0E12FF0E0EE5FFB4F85E396E06081F3
:102DE0000E94B52E1F5F80916704181790F385E34A
:102DF00096E060E20E94B52E85E396E06DE00E94C9
:102E0000B52E10E00AC0E12FF0E0EE5FFB4F85E346
:102E100096E060810E94B52E1F5F809167041817AD
:102E200090F31CC08B3119F40E94C6161FC08D3060
:102E3000E9F08A30D9F080916704843688F485E31C
:102E400096E0612F0E94B52E80916704E82FF0E094
:102E5000EE5FFB4F10838F5F8093670480E007C0B5
:102E600085E396E067E00E94692BF8CF81E01F912F
:102E700008951F93CF93DF93CFEDD3E010E03BC0D5
:102E800085E396E062E271E00E94FA2C85E396E029
:102E9000612F4AE050E00E94772C85E396E06FE2D4
:102EA00071E00E94FA2C699170E080E090E020913E
:102EB000DE0330E040E050E00E94492F20E137E29D
:102EC00040E050E00E94492FDC01CB014091D50346
:102ED0005091D6036091D7037091D803480F591FC2
:102EE0006A1F7B1F85E396E02AE030E00E943E2CBB
:102EF0001F5F183119F08881882311F6DF91CF9177
:102F00001F910895EF92FF920F931F93882339F436
:102F100085E396E061E77AE00E94872B3BC090E072
:102F20000E94B20824E630E040E050E00E947B2F8F
:102F3000122F032FF42EE52E622F732F842F952F3F
:102F40002AE030E040E050E00E947B2F85E396E0ED
:102F5000BA01A9012AE030E00E942F2C85E396E017
:102F60006EE20E94692B612F702F8F2D9E2D2AE01B
:102F700030E040E050E00E947B2FAB01BC0185E3D4
:102F800096E02AE030E00E942F2C85E396E063E78C
:102F90000E949B2B1F910F91FF90EF900895FF923D
:102FA0000F931F93CF93DF9385E396E067E67AE074
:102FB0000E94482B8091B503813041F485E396E06F
:102FC0006EE47AE00E94872BFF246DC0823029F4E2
:102FD00085E396E067E37AE0F5CF843029F485E372
:102FE00096E063E27AE0EECF853071F785E396E014
:102FF00068E17AE0E7CFCF2DD0E0C930D1051CF0F1
:103000006F2D685C02C06F2D6F5C85E396E00E94B7
:10301000692B85E396E060E17AE00E94482BBE01CF
:103020006F5F7F4F85E396E04AE050E00E94D32C2B
:1030300085E396E065E07AE00E94482B8E010B5410
:103040001C4FD8011196EC91E032F8F485E396E03C
:1030500068EF79E00E94482BF8018181803130F0DF
:1030600085E396E063E371E00E94FA2CCB54DC4FD9
:10307000698170E06F7070706F5F7F4F85E396E0DD
:103080004AE050E00E94E62C0DC0F0E0EF70F070D6
:10309000EE0FFF1FE75BFC4F6081718185E396E0D7
:1030A0000E94FD2CF39480918A04F81608F4A3CFB3
:1030B00085E396E06DED79E00E94482B8091CD0389
:1030C0000E94821785E396E062EC79E00E94482B2B
:1030D0008091CE030E94821785E396E067EA79E04B
:1030E0000E94482B8091CF030E94821785E396E0CF
:1030F0006CE879E00E94482B4091C5035091C603CB
:103100006091C7037091C8034115510561057105B0
:1031100039F185E396E02AE030E00E943E2C85E319
:1031200096E069E579E00E94482B8091C9030E94EE
:10313000E508AB01BC0185E396E02AE030E00E949F
:103140003E2C85E396E065E379E00E94482B85E319
:1031500096E06091CA034AE050E00E94892C06C0C4
:1031600085E396E06CE279E00E94872B85E396E0A8
:103170006FE079E00E94482B6091CB037091CC0303
:1031800085E396E04AE050E00E94632C85E396E0F8
:1031900062EF78E00E94482B6091C403603450F4E1
:1031A00070E06F5F7F4F85E396E04AE050E00E9459
:1031B000E62C06C085E396E069EE78E00E94872B56
:1031C00085E396E06CEC78E00E94482B8091C30385
:1031D00080FD03C065E371E002C069E371E085E34F
:1031E00096E00E94FD2C85E396E06FEA78E00E946D
:1031F000482B8091C30382700E94930D85E396E073
:1032000060E978E00E94482B8091C30384700E949B
:10321000930D85E396E061E778E00E94482B80916A
:10322000C30388700E94930DCDB7DEB7E5E00C9420
:10323000E12F1F93CF93DF9385E396E06BEB7BE069
:103240000E94482B4091D5035091D6036091D7033B
:103250007091D80385E396E02AE030E00E943E2C8E
:1032600085E396E065EA7BE00E94482B4091D90314
:103270005091DA036091DB037091DC0385E396E003
:1032800020E130E00E943E2C85E396E06FE87BE091
:103290000E94482B85E396E06091DD034AE050E010
:1032A0000E94892C85E396E069E77BE00E94482B29
:1032B00085E396E06091DE034AE050E00E94892CAD
:1032C00085E396E063E67BE00E94482BCFEDD3E0F8
:1032D00010E012C0112331F085E396E06DE371E058
:1032E0000E94FA2C85E396E069914AE050E00E9442
:1032F000772C1F5F183119F08881882359F785E3EF
:1033000096E00E94712B85E396E06DE47BE00E94DD
:10331000482B85E396E06091F7034AE050E00E9475
:10332000892C85E396E068E37BE00E94482BE091DE
:10333000F803F0E0E770F070EE0FFF1FE759FC4F65
:103340006081718185E396E00E94FD2C85E396E023
:1033500063E27BE00E94482B8091F80390E0887143
:1033600090708830910589F0893091051CF4892B83
:1033700039F01BC08031910569F04897B1F40FC056
:1033800085E396E06AE17BE00EC085E396E06EE0BF
:103390007BE009C085E396E068E07BE004C085E35C
:1033A00096E06EEF7AE00E94872B85E396E06AEE66
:1033B0007AE00E94482B4091D1035091D203609152
:1033C000D3037091D40385E396E02AE030E00E94B5
:1033D0003E2C85E396E061ED7AE00E94482B8091D7
:1033E000A10380710E94930D85E396E068EB7AE07B
:1033F0000E94482B8091A10380740E94930D85E365
:1034000096E06FE97AE00E94482B8091A1038072D8
:103410000E94930D85E396E062E87AE00E94482BD3
:1034200080ED93E00E94F508AB01BC0185E396E0D6
:103430002AE030E00E942F2C85E396E06DE77AE0E9
:103440000E94482B80ED93E00E94F5089B01AC019F
:1034500060E472E48FE090E00E947B2F85E396E0C9
:10346000BA01A9012AE030E00E942F2C85E396E002
:103470006AE77AE00E94872BDF91CF911F91089530
:10348000EF92FF920F931F937C0105E316E0C801B2
:103490006F2D70E04AE050E00E94522CC8016EE2AD
:1034A0000E94692BB70184E0769567958A95E1F7CC
:1034B0006F707070C8014AE050E00E94522CC80141
:1034C0006EE20E94692B8FE0E822FF24C801B70159
:1034D0004AE050E00E94522C1F910F91FF90EF9014
:1034E00008950F931F93CF93DF93209101042F3FF3
:1034F000A9F585E396E061EF75E00E94482B81E72E
:1035000093E00E94401A85E396E060ED75E00E942A
:10351000482B80918B0490918C040E94401A85E383
:1035200096E06DE975E00E94872B85E396E06AE7F7
:1035300075E00E94872B85E396E062E675E00E94C5
:10354000872B85E396E06DE375E00E94872B85E38A
:1035500096E00E94712B0E94CF1769C012160CF0E2
:1035600066C0332727FD309580918A0490E082174A
:1035700093070CF45CC085E396E068E275E00E9476
:10358000482B60910104772767FD709585E396E0ED
:103590004AE050E00E94E62C85E396E06DEF74E08F
:1035A0000E94482B08E210E03AC0C12FD0E0CC0FB7
:1035B000DD1FC759DB4F288130E080910104992736
:1035C00087FD909501972817390741F585E396E027
:1035D0006FE371E00E94FA2C85E396E0602F4AE0E9
:1035E00050E00E94772C85E396E063E471E00E944E
:1035F000FA2CE981F0E0EF70F070EE0FFF1FE75B4F
:10360000FC4F6081718185E396E00E94FA2C85E38E
:1036100096E067E471E00E94FA2C0F5F1F5F8091D3
:103620008904181710F285E396E00E94712BDF9150
:10363000CF911F910F910895ACE1B0E0E2E2FBE180
:103640000C94C22F282F809101048F3F09F042C1B2
:10365000822F90E0FC013A97EF36F10508F033C174
:10366000EC5CFF4F0C94EF2F85E396E069E471E08A
:10367000AEC085E396E069E471E00E94FD2C1CC1B8
:1036800085E396E065E571E00E94FD2C85E789837E
:10369000DE011296E5EBF3E08BE101900D92815093
:1036A000E1F7CE0101966CE10E94D70F0E947C0CDD
:1036B00083E080939A0368EC70E080E090E00E94E1
:1036C000D42980919A03843009F0FDC08FE70E94CD
:1036D000930A0E94A70A8983853509F0F4C085E31F
:1036E00096E06FED74E00E94872B85E396E061EC35
:1036F00074E00E94872B85E396E063EA74E0ACC037
:1037000085E396E06DE671E00E94FD2C89E68983F1
:10371000CE01019661E00E94D70F0E947C0C83E0ED
:1037200080939A0368EC70E080E090E00E94D429D6
:1037300080919A03843009F0C6C08FE70E94930AF3
:103740000E94A70A89838E010E5F1F4FBDE1EB2EF9
:10375000F12CEC0EFD1E0E94A70AD8018D938D015D
:10376000AE15BF05C1F7A5EBB3E0FE0132968BE1C4
:1037700001900D928150E1F78981893409F0A3C04D
:1037800085E396E065E874E00E94872B85E396E088
:1037900067E674E00E94872B85E396E069E474E0B5
:1037A0005BC085E396E067E871E00E94FD2C8EEF38
:1037B0008093010488C020522750922F905380910B
:1037C0008A04891738F485E396E066E971E00E947F
:1037D000FD2C79C0909301046FC084E180930104B3
:1037E00085E396E062E174E037C085E180930104EF
:1037F00085E396E06BED73E02FC086E180930104D2
:1038000085E396E064EA73E027C087E180930104D2
:1038100085E396E06AE573E01FC088E180930104C8
:1038200085E396E069E473E017C089E180930104C1
:1038300085E396E065E373E00FC08AE180930104BD
:1038400085E396E060E273E007C08BE180930104BA
:1038500085E396E068EF72E00E94872B34C085E331
:1038600096E06EED72E00E94872B8091C30391E099
:103870001DC085E396E068EC72E00E94872B809182
:10388000C30392E013C085E396E063EB72E00E940D
:10389000872B8091C30394E009C085E396E068E933
:1038A00072E00E94872B8091C30398E08927809360
:1038B000C3038FEF809301040E94711A04C085E353
:1038C00096E00E947C2E85E396E00E94422E892B92
:1038D000B1F762C1822F0E94D016882309F45CC11F
:1038E00080916704882321F48FEF809301044CC1F9
:1038F00082E094E060E070E040E050E00E94A206C8
:103900009B01AC0160910104862F992787FD90955A
:10391000A92FB92FFC013197EB31F10508F024C133
:10392000ED55FF4F0C94EF2FE62FFF27E7FDF095A5
:1039300080918A0490E08E179F070CF415C1DA017C
:10394000C9010197A109B1098097A105B10548F006
:10395000A8E2FA2E00E010E06F010894C108D10837
:1039600025C0EB54FC4F822F81508083E5C0612F2E
:1039700070E0660F771F67597B4FFB01808190E0F5
:103980008C159D0591F48F2D90E0A0E0B0E082179A
:103990009307A407B50741F4F601EB54FC4FDB0194
:1039A00011968C91818301E0F3941F5F80918904CB
:1039B0001817E8F2BFC02F3F31054105510511F03E
:1039C00008F0D2C02093CD03B7C02F3F3105410589
:1039D000510511F008F0C8C02093CE03ADC02F3FB1
:1039E00031054105510511F008F0BEC02093CF0309
:1039F000A3C0809102048062803719F583E094E0CF
:103A000060E070E040E050E00E94A2069B01AC0143
:103A1000DC01CB010197A109B1090897A105B10506
:103A200008F0B5C0CA01B90124ED30E340E050E030
:103A30000E94492F9B01AC012A5E3C4A4A46554EE2
:103A400024C0863611F583E094E060E070E040E049
:103A500050E00E94A2069B01AC01DC01CB01019762
:103A6000A109B1090797A105B10508F090C0CA01E5
:103A7000B90128EA31E640E050E00E94492F9B015D
:103A8000AC01245E3C434E46544E211531054105A0
:103A9000510561F0DA01C901805C9D49A845B54333
:103AA00081509A45A246B24008F05EC02093C503FB
:103AB0003093C6034093C7035093C8033DC02F3FC4
:103AC00031054105510511F008F04EC02093C9039E
:103AD00033C0DA01C9010197A109B1098F3F9105EE
:103AE000A105B10508F040C02093CA0325C0DA0142
:103AF000C901845C9940A040B0408D549D41A040D4
:103B0000B04030F43093CC032093CB0301E001C0EC
:103B100000E0211531054105510511F48FEF07C073
:103B2000213431054105510528F4822F81508093BD
:103B3000C40302C00023C1F0809168048823D1F43B
:103B40008091D9039091DA03A091DB03B091DC035B
:103B50000196A11DB11D8093D9039093DA03A09320
:103B6000DB03B093DC0306C085E396E068EA71E00E
:103B70000E94FD2C0E94C6168FEF8093010485E3FE
:103B800096E06AE00E949B2B0E94711A05C021E01A
:103B900030E040E050E07ECF6C96E8E00C94DE2F01
:103BA00085E396E06CE472E00E94872B85E396E063
:103BB00064E372E00E94872B85E396E00E94422E28
:103BC000892B31F085E396E00E947C2E0E941C1B1D
:103BD0000E94DF14823019F0833069F405C085E358
:103BE00096E066E172E004C085E396E06FEF71E075
:103BF0000E94872B08958FEF809301041092680430
:103C00000E94711A0CC085E396E00E94422E892B17
:103C100031F085E396E00E947C2E0E941C1B80916F
:103C200001048E3F81F7089580910104992787FD53
:103C30009095A92FB92FFC013196EB30F10508F0D2
:103C400074C0E254FF4F0C94EF2F85E396E064E6D6
:103C500078E00E94872B81E793E00E94401A85E379
:103C600096E06CE478E00E94872B85E396E067E2BB
:103C700078E00E94872B85E396E06DEF77E00E9465
:103C8000872B85E396E06CED77E00E94872B85E338
:103C900096E06FEA77E00E94872B85E396E069E87B
:103CA00077E00E94872B85E396E065E677E00E9447
:103CB000872B85E396E06EE377E00E94872B85E310
:103CC00096E00E94712B0E9419192FC085E396E09F
:103CD00061E277E028C085E396E06CEF76E023C0F0
:103CE00085E396E067EE76E01EC085E396E068EC3B
:103CF00076E019C085E396E064E876E014C085E3D9
:103D000096E06FE676E00FC085E396E06AE576E040
:103D10000E94872B85E396E064E176E004C085E3AA
:103D200096E06EEF75E00E94872B6AE070E080E01D
:103D300090E00E94D42904C085E396E00E947C2E86
:103D400085E396E00E94422E892BB1F70895A2E206
:103D5000B0E0EDEAFEE10C94B82F8E010F5F1F4F2B
:103D600080E1D8011D928A95E9F785E396E066EC3B
:103D700071E00E94FD2C0E948B1520EC3DE948E586
:103D800055E32F8F38A349A35AA380EC97EFAAEBF2
:103D9000B7E38B8F9C8FAD8FBE8F24EF31E040E077
:103DA00050E02F8B388F498F5A8F30E5C32E33EC7C
:103DB000D32EE12CF12C20EC422E2DE9522E28E5B9
:103DC000622E25E3722E88249924540133241E8AFE
:103DD0001D8A198A1A8A1B8A1C8AFFC085E396E00D
:103DE0000E947C2E8434B9F0853430F48332B9F1EA
:103DF0008C3209F0CCC044C0833509F0C8C02F8D87
:103E000038A149A15AA1C901DA012C013D01882438
:103E100099245401E2C085E396E064E40E94692B92
:103E200085E396E040EC5DE968E575E32AE030E083
:103E30000E949D2C85E396E06CE20E94692B85E34D
:103E400096E040EC57EF6AEB77E32AE030E00E941F
:103E50009D2C85E396E06CE20E949B2BBEC01982EC
:103E60001A821B821C821D821E821F82188619865E
:103E70001A861B861C861D861E861F86188A3AC0D7
:103E8000339434E0331609F0A8C069817A818B81BC
:103E90009C8128EE33E040E050E00E94492F6F8F74
:103EA00078A389A39AA36D817E818F8198850E94D2
:103EB000492F6B8F7C8F8D8F9E8F89859A85AB85DF
:103EC000BC858F8B988FA98FBA8F6D857E858F85E6
:103ED00098890E94492F6B017C0190E2C9169EE4EB
:103EE000D90690E0E90690E0F90630F48CE162E34F
:103EF0000E94BD0A332471C0A0E3CA16A5E7DA0602
:103F0000A0E0EA06A0E0FA0618F48CE162E2F0CF45
:103F1000B0E4CB16BCE9DB06B0E0EB06B0E0FB0694
:103F200018F48CE166E2E4CFE0E5CE16E3ECDE06C1
:103F3000E0E0EE06E0E0FE0618F48CE162E1D8CFA6
:103F4000F0E6CF16FAEEDF06F0E0EF06F0E0FF064F
:103F500018F48CE165E1CCCF20E7C21621E1D2064E
:103F600021E0E20620E0F20618F48CE161E0C0CF27
:103F700030EAC31636E8D30631E0E30630E0F30654
:103F800018F48CE163E0B4CF8CE165E0B1CF90ED43
:103F9000292E280E49E0421500F1032D10E0000FF4
:103FA000111F000F111F81E090E08C0F9D1F080F63
:103FB000191FD8016D917D918D919C912AE030E07F
:103FC00040E050E00E94492F620D711D811D911D3E
:103FD000F801608371838283938385E396E00E9476
:103FE000422E892B09F0FACE81149104A104B10468
:103FF00089F4C301B2010E94330B61E070E080E0FC
:1040000090E00E94D429FFEFFE8B1D8A198A1A8A3C
:104010001B8A1C8A2F89388D498D5A8D82169306EA
:10402000A406B506E0F40E94DE0A29893A894B8984
:104030005C89280F311D411D511D298B3A8B4B8BFB
:104040005C8B3D89381708F48D8B4E89841708F4F2
:104050008E8B0894811C911CA11CB11C56C0C301FD
:10406000B20128EE33E040E050E00E947B2F85E370
:1040700096E0BA01A9012AE030E00E942F2C85E3E6
:1040800096E06CE20E94692B85E396E06D894AE038
:1040900050E00E94772C85E396E06CE20E94692B49
:1040A00069897A898B899C89A50194010E947B2F5B
:1040B00085E396E0BA01A9012AE030E00E942F2CA6
:1040C00085E396E06CE20E94692B85E396E06E89B9
:1040D0004AE050E00E94772C85E396E06CE20E9473
:1040E0009B2B4C0C5D1C6E1C7F1C8B8D9C8DAD8D99
:1040F000BE8D84159505A605B70520F44F8C58A0F4
:1041000069A07AA08824992454012F8D38A149A14F
:104110005AA1285E33404040504009F05ECFA2963D
:10412000E2E10C94D42FAAE5B0E0E9E9F0E20C94C6
:10413000C42F8B017A018B3009F426C18C3040F5F5
:10414000853009F484C0863080F4823009F459C087
:10415000833020F4813009F050C242C0833009F42A
:1041600061C0843009F049C265C0883009F49DC03F
:10417000893038F4863009F486C0873009F03DC2B2
:104180008CC0893009F499C08A3009F036C2C9C0A0
:10419000893609F482C18A3680F4863609F42DC145
:1041A000873620F4853609F028C20EC1873609F417
:1041B0003DC1883609F021C241C18C3609F4C4C121
:1041C0008D3638F48A3609F473C18B3609F015C27E
:1041D000AFC18D3609F4ECC1873C09F00EC200C2B4
:1041E00081E069E270E00E948F1100ED13E0F801B8
:1041F00081918F010E947811F3E0093F1F07B9F701
:1042000004C282E06BE170E00E948F1105EB13E0C5
:10421000F80181918F010E947811F3E0003D1F07A2
:10422000B9F7F3C183E061E070E00E948F110E9452
:10423000DF14E9C184E061E070E00E948F1181E049
:104240000E9478110E9471110E94A71EE0C1609126
:10425000890470E0660F771F85E00E948F1100E0EF
:1042600010E008C0F801E759FB4F80810E947811E7
:104270000F5F1F4F8091890490E0880F991F0817E6
:10428000190780F3C2C186E062E070E00E948F11DE
:1042900081E793E00E948611B8C187E061E070E099
:1042A0000E948F1180918A04AEC188E061E070E0C5
:1042B0000E948F1180919B03A6C186E68983CE015F
:1042C000019661E00E94D70F0E947C0C83E08093EE
:1042D0009A0368EC70E080E090E00E94D42980911D
:1042E0009A038430E1F48FE70E94930A0E94A70AA0
:1042F0008983863471F489E060E270E00E948F1156
:1043000010E00E94A70A0E9478111F5F1032C9F7BF
:104310007CC189E061E070E00E948F11C7C089E034
:104320006DC18AE069E170E00E948F1182E08093A4
:104330009C0380919F05882351F08091A103909167
:10434000A203A091A303B091A403806809C0809147
:10435000A1039091A203A091A303B091A4038F772E
:104360008093A1039093A203A093A303B093A4030B
:104370000CE913E0F80181918F010E947811F3E0BC
:10438000053B1F07B9F741C18BE061E270E00E9475
:104390008F118091BE048F3F39F08091BE048F5FF2
:1043A0008093BE04815002C08091BE040E947811A7
:1043B00010E0812F0E94AE110E94190A0E948611FE
:1043C0001F5F1031B1F721C185E661E070E00E9406
:1043D0008F110932110509F015C120E030E0F90113
:1043E000E053FC4FD701A20FB31F8C9180832F5F46
:1043F0003F4F2932310599F759C086E661E070E0F8
:104400000E948F110B31110509F0FCC020E030E053
:10441000F901EB54FC4FD701A20FB31F8C9180839D
:104420002F5F3F4F2B31310599F740C087E661E0A0
:1044300070E00E948F110E94881638C088E661E003
:1044400070E00E948F1185E78A83DE011396E5EB09
:10445000F3E08BE101900D928150E1F7CE010296DD
:104460006CE10E94D70F0E947C0C83E080939A033A
:1044700060E273E080E090E00E94D42980919A038A
:10448000843009F0BFC08FE70E94930A0E94A70AF8
:104490008A83853509F0B6C009C089E661E070E01D
:1044A0000E948F110E944D080E94920881E0ABC0CB
:1044B0008AE661E070E00E948F1189E68E8FCE015E
:1044C0004E9661E00E94D70F0E947C0C83E080939F
:1044D0009A0360E273E080E090E00E94D42980912A
:1044E0009A03843009F08EC08FE70E94930A0E94DD
:1044F000A70A8E8F8E01015E1F4F4AE3E42EF12C36
:10450000EC0EFD1E0E94A70AF80181938F01EE15A3
:10451000FF05C1F7A5EBB3E0FE017F968BE10190AB
:104520000D928150E1F78E8D893409F06BC0BECFBA
:104530008BE661E070E00E948F11F70180810E949C
:10454000B6160E949116B2CF8CE661E070E00E9430
:104550008F110032110571F487E68AAFDE01DB9618
:10456000F70180E201900D928150E1F7CE01CA96E9
:1045700061E205C087E48AAFCE01CA9661E00E947D
:10458000D70F0E947C0C83E080939A036CE474E064
:1045900080E090E00E94D42980919A03843091F5C4
:1045A0008FE70E94930A0E94A70A873459F57ECFAD
:1045B0008DE661E070E00E948F110931110511F55F
:1045C00020E030E0F901E456FC4FD701A20FB31F01
:1045D0008C9180832F5F3F4F2931310599F766CF4A
:1045E00087EC61E070E00E948F1181E00E947811F9
:1045F0000E9471111092FF030AC08AEC61E070E022
:104600000E948F1180E00E9478110E947111C65A99
:10461000DF4FE6E00C94E02FA0E0B0E0E2E1F3E24F
:104620000C94C02F84E0A82E06E0B02E15E0C12E19
:1046300003E315E0B4E6DB2EA2E0EA2EF3E0FF2E62
:10464000A1C085E396E00E947C2E982F80939E0562
:1046500080919D05833021F1843028F4813099F0D8
:104660008230B8F409C0853009F448C0853020F1A3
:10467000863009F087C05FC0953B09F083C081E0B8
:1046800080939D057FC0923609F07AC0E0929D0527
:1046900079C090939C0590939B05F0929D0572C004
:1046A0009093990510929A0580919B058927809394
:1046B0009B05A0929D0566C0D92FC0E02091990569
:1046C00030919A052C2B3D2B30939A052093990518
:1046D00080919B05892780939B05C0929D05253677
:1046E000310508F44FC08CEC61E070E00E948F113E
:1046F00081E00E9478110E94711142C020919705BB
:1047000030919805F901ED5CFA4F908380919B05FB
:10471000892780939B052F5F3F4F30939805209307
:1047200097058091990590919A052817390750F1BE
:10473000B0929D0527C080919B05891759F460911F
:1047400097057091980580919C0543E355E00E9480
:1047500093200DC08BEC62E070E00E948F1180917D
:104760009C050E947811809100040E947811F80144
:104770008D2D11928A95E9F7109298051092970560
:1047800010929D0585E396E00E94422E892B09F048
:1047900058CFCDB7DEB7EAE00C94DC2F81E08093F0
:1047A000FF0308C085E396E00E94422E892B11F09A
:1047B0000E940C238091FF038823A1F70895A0E0B5
:1047C000B0E0E5EEF3E20C94C32F0E94AE29611530
:1047D000710581059105C9F30E9499061092D903CC
:1047E0001092DA031092DB031092DC03DD24E090D8
:1047F000D903F090DA030091DB031091DC03102F52
:104800000F2DFE2CEE240E9494062FEF30E040E0A6
:1048100050E00E949D2FE60EF71E081F191FE09220
:10482000D903F092DA030093DB031093DC03D394F3
:1048300044E0D416E1F6CFEDD3E000E010E090E1E3
:10484000E92E97E2F92E4EC00F5F19F40E944D0831
:104850004DC00E94940622E330E040E050E00E9408
:104860009D2F6F5FEFEDF3E090E004C0819186171C
:1048700059F39F5F9117D0F38091DE0390E08E9DF6
:1048800090018F9D300D9E9D300D1124862F90E05C
:10489000AC01249FC001259F900D349F900D1124E1
:1048A000AA2797FDA095BA2F2091D5033091D60362
:1048B0004091D7035091D803820F931FA41FB51FB7
:1048C00020919D0330919E0340919F035091A0033E
:1048D000281739074A075B0708F4B6CF69931F5FAB
:1048E000183121F08881882309F0AECFCDB7DEB72B
:1048F000E7E00C94DF2F1F93109101041F3F09F094
:10490000F1C0893409F467C08A3428F5883309F482
:1049100079C0893368F4803309F486C0813308F0A4
:104920006FC08B3109F44DC0813209F0D5C03DC054
:10493000813409F49AC0823438F4893309F472C09E
:10494000803409F0C9C031C0823409F4A1C0863472
:1049500009F0C2C052C0823609F49AC0833690F47E
:10496000883579F1893538F4823509F43FC08335CB
:1049700009F0B2C01FC08A3509F4A9C0813609F018
:10498000ABC073C0823791F1833730F48636A9F11A
:10499000893609F0A1C01FC0883799F08A3709F419
:1049A00096C0833709F098C005C085E396E069E4B6
:1049B00071E019C00E94881685E396E063ED71E00E
:1049C00006C00E94911685E396E06DEE71E00E94AC
:1049D000FD2C8EEF7FC00E944D080E94920885E357
:1049E00096E06CE072E00E94FD2C76C00E94DF230E
:1049F00085E396E065E272E0F6CF0E9439176CC05D
:104A0000805368C085E396E06CEE71E00E94872BCE
:104A10009091F803892F885F8871977E892B809306
:104A2000F80320C089E056C085E396E069ED71E0A7
:104A30000E94872B8091A1039091A203A091A303D0
:104A4000B091A40320E130E040E050E082279327BA
:104A5000A427B5278093A1039093A203A093A30357
:104A6000B093A4031093010437C085E396E063EC90
:104A700071E00E94872B8091A1039091A203A091E5
:104A8000A303B091A40320E430E040E050E012C062
:104A900085E396E062EB71E00E94872B8091A10391
:104AA0009091A203A091A303B091A40320E230E06F
:104AB00040E050E082279327A427B5278093A103E5
:104AC0009093A203A093A303B093A40302C00E94F7
:104AD000D01D8FEF80930104809101048E3F09F473
:104AE000DDC0D4C00E94D016882309F4D7C08091BD
:104AF0006704882321F48FEF80930104C7C082E00C
:104B000094E060E070E040E050E00E94A2069B016B
:104B1000AC0180910104992787FD9095A92FB92FA9
:104B2000FC013197E930F10508F08CC0E753FF4FE5
:104B30000C94EF2FDA01C901815C9D49A845B5436A
:104B40008F5F9945A246B24008F07CC02093D50300
:104B50003093D6034093D7035093D8039AC0209341
:104B6000D9033093DA034093DB035093DC0381E0F5
:104B7000809368048EC0283031054105510508F046
:104B800061C02093DD0385C0DA01C9010197A10945
:104B9000B1090A97A105B10508F054C02093DE03BE
:104BA00078C082E094E06DE371E00E94BE0710E0FF
:104BB0000EC0183130F4E12FF0E0E053FC4F87874E
:104BC0001F5F80E090E06DE371E00E94BE070097F8
:104BD00059F00E94A007009761F706C0E12FF0E0AE
:104BE000E053FC4F17861F5F1831C0F352C02530C9
:104BF00031054105510530F52093F7034AC0DA012C
:104C0000C9010197A109B1090697A105B105D0F421
:104C10008091F803887F822B8093F8033AC0DA01F1
:104C2000C9010197A109B1098050924CA140B0403F
:104C300048F42093D1033093D2034093D30350938D
:104C4000D40327C085E396E068EA71E00E94FD2C5A
:104C500013C08091D9039091DA03A091DB03B09146
:104C6000DC030196A11DB11D8093D9039093DA0353
:104C7000A093DB03B093DC030E94C6168FEF8093F2
:104C8000010485E396E06AE00E949B2B0E94141EBB
:104C900005C0809168048823E1F2EECF1F9108954A
:104CA0008FEF80930104109268040E94141E0CC0C0
:104CB00085E396E00E94422E892B31F085E396E051
:104CC0000E947C2E0E947B24809101048E3F81F7FC
:104CD0006AE070E080E090E00E94D42904C085E39F
:104CE00096E00E947C2E85E396E00E94422E892B5E
:104CF000B1F70895AAE2B0E0E0E8F6E20C94BD2F27
:104D00000E94A0297B018C0181E00E949D0B04C0C0
:104D100085E396E00E947C2E85E396E00E94422E79
:104D2000892BB1F72D98DD24D39452E6752E42E0FD
:104D3000842E912C8C0E9D1E5E010894A11CB11C2A
:104D400033E0C32E0E94A02920E030E06E197F09D5
:104D5000800B910B693C71058105910510F021E0F4
:104D600030E08D2D90E028233923232B99F10E94E8
:104D7000A0297B018C012C9A80ED97E00E94E41120
:104D80007982D401E0EDF3E089E201900D92815047
:104D9000E1F7C5016AE20E94D70F2C9880E090E00D
:104DA0000E94E411C0929A030E947C0C62E370E0BE
:104DB00080E090E00E94D42980919A03843051F4DD
:104DC000C0929A038FE70E94930A0E94A70A823436
:104DD00009F4DD248BE00E94D22A892B49F5DD24D9
:104DE000D39426C02D9A2C9A85E396E00E947C2EBF
:104DF0008D30910569F08E3091051CF40A97B1F45D
:104E000007C08332910569F08234910579F40CC0B2
:104E100085E396E064EA71E00E94872B0E945026A9
:104E200005C00E94A71E02C00E94CE232D982C9878
:104E300085E396E00E94422E892B09F483CFD2CFDE
:104E40008F929F92AF92BF92CF92DF92EF92FF929A
:104E50000F931F938BE00E94D22A892B09F083C005
:104E600068EC70E080E090E00E94D42980E090E05F
:104E70000E94E4110E94A0295B016C0160ECE62E07
:104E800062E1F62E012D112DEA0CFB1C0C1D1D1DDF
:104E900006C08BE00E94D22A892B09F062C00E94D2
:104EA000A0296E157F058007910798F38BE00E947B
:104EB000D22A892B09F055C080ED97E00E94E411B9
:104EC0000E94A0297B018C0199249394882488E472
:104ED00096E2A0E0B0E0A80EB91ECA1EDB1E29C0F3
:104EE000AE14BF04C006D10638F480ED97E00E94EE
:104EF000E411882483941DC00E94A0296E197F09A3
:104F0000800B910B693C71058105910590F00E9421
:104F1000A0297B018C0180E0992009F481E0982E82
:104F2000882319F480E090E002C080ED97E00E94B1
:104F3000E4118BE00E94D22A892B91F280E090E06C
:104F40000E94E411882049F080919B038F5F837059
:104F50000E94B6160E94911606C00E94DF230E948E
:104F600088160E947A261F910F91FF90EF90DF9094
:104F7000CF90BF90AF909F908F90089580E06DEF9D
:104F800077E042E050E00E94DB280895EF92FF9224
:104F90000F931F9380E00E9419080E94CF118DE0AB
:104FA00061E00E94332A8CE061E00E94332A8BE0AA
:104FB00060E00E94332A83E060E00E94332A83E0AD
:104FC00061E00E949F2A8EE061E00E94332A8EE019
:104FD00060E00E949F2A0E94B71485E396E040E0BB
:104FE00052EC61E070E00E94BB2D0E94A9160E9465
:104FF00091160E94720D8FEF8093BE040E94BE270F
:1050000078940E94A0297B018C018091BE048F3F7F
:1050100009F0C7C00E94A0296E197F09800B910B6F
:10502000605D77408040904008F0BBC0EECF85E3E4
:1050300096E00E947C2E85E396E00E94422E892B0A
:10504000B1F785E396E062E472E00E94FA2C81E712
:1050500093E00E94401A85E396E069E572E00E94C1
:10506000FA2C85E396E062E070E04AE050E00E94AE
:10507000E62C62E370E080E090E00E94D42985E3B2
:1050800096E00E94422E04970CF185E396E00E9480
:105090007C2E82349105D1F485E396E00E947C2E2B
:1050A0008E34910599F485E396E00E947C2E843439
:1050B000910561F485E396E00E947C2E819731F49E
:1050C00080E090E00E94E4110E947A264091D10392
:1050D0005091D2036091D3037091D403DB01CA01D4
:1050E0000197A109B1090497A105B10568F440939E
:1050F000BF04433029F040E052EC61E070E004C0AE
:1051000040EA56E861E070E085E396E00E94BB2D3E
:105110000E9420272D9880E090E00E94E4110E94D8
:10512000720D80E00E949D0B8091A4040E94C80A29
:105130000E947C0C109227051092280510922905D8
:1051400010E015C062E370E080E090E00E94D42996
:1051500080ED97E00E94E41162E370E080E090E06F
:105160000E94D42980E090E00E94E4111F5F8091AA
:105170009B03811738F78091F80390E084FF09C002
:1051800020E088719070489709F421E0822F0E94F6
:10519000C0148FE00E9419081F910F91FF90EF90AB
:1051A000089580ED97E00E94E4118BE061E00E9499
:1051B0009F2A2D9A40CF823000F5E82FF0E0EE0FC5
:1051C000FF1FE056FA4F71836083882319F0813006
:1051D000A1F408C0809169008C7F842B80936900C2
:1051E000E89A089580916900440F551F440F551F98
:1051F000837F842B80936900E99A08951F920F9210
:105200000FB60F9211242F933F934F935F936F9399
:105210007F938F939F93AF93BF93EF93FF9380916F
:10522000A0059091A105892B29F0E091A005F091AE
:10523000A1050995FF91EF91BF91AF919F918F913A
:105240007F916F915F914F913F912F910F900FBE82
:105250000F901F9018951F920F920FB60F92112466
:105260002F933F934F935F936F937F938F939F936E
:10527000AF93BF93EF93FF938091A2059091A30505
:10528000892B29F0E091A205F091A3050995FF91E2
:10529000EF91BF91AF919F918F917F916F915F91AE
:1052A0004F913F912F910F900FBE0F901F90189527
:1052B0001F920F920FB60F9211242F933F938F934B
:1052C0009F93AF93BF938091A8059091A905A0915A
:1052D000AA05B091AB053091AC050196A11DB11D99
:1052E000232F2D5F2D3720F02D570196A11DB11DC5
:1052F0002093AC058093A8059093A905A093AA05D7
:10530000B093AB058091A4059091A505A091A60549
:10531000B091A7050196A11DB11D8093A40590939E
:10532000A505A093A605B093A705BF91AF919F9146
:105330008F913F912F910F900FBE0F901F90189556
:105340008FB7F8942091A8053091A9054091AA053E
:105350005091AB058FBFB901CA0108959FB7F8946A
:105360002091A4053091A5054091A6055091A7056F
:1053700086B5A89B06C08F3F21F02F5F3F4F4F4F50
:105380005F4F9FBF542F432F322F2227280F311DED
:10539000411D511D82E0220F331F441F551F8A9566
:1053A000D1F7B901CA010895EF92FF920F931F93AD
:1053B000CF93DF937B018C010E94AE29EB010EC0DD
:1053C0000E94AE296C1B7D0B685E7340C8F3089485
:1053D000E108F10801091109C851DC4FE114F10499
:1053E0000105110569F7CDB7DEB7E6E00C94E02FB3
:1053F000789484B5826084BD84B5816084BD85B5B0
:10540000826085BD85B5816085BDEEE6F0E0808176
:1054100081608083E1E8F0E0108280818260808397
:10542000808181608083E0E8F0E08081816080831A
:10543000E1EBF0E0808184608083E0EBF0E080814C
:1054400081608083EAE7F0E08081846080838081EE
:105450008260808380818160808380818068808396
:105460001092C1000895CF93DF93482F50E0CA01F6
:105470008D5F934FFC0134914151544FFA01849157
:10548000882369F190E0880F991FFC01EF52F44FD7
:10549000A591B491FC01E552F44FC591D4916623D6
:1054A00051F42FB7F8948C91932F909589238C9376
:1054B000888189230BC0623061F42FB7F8948C91F6
:1054C000932F909589238C938881832B88832FBF7A
:1054D00006C09FB7F8948C91832B8C939FBFDF916C
:1054E000CF910895833071F0843028F48130A1F099
:1054F000823021F514C08630B1F08730D1F084308D
:10550000E9F404C0809180008F7703C0809180000F
:105510008F7D80938000089584B58F7702C084B515
:105520008F7D84BD08958091B0008F778093B00007
:1055300008958091B0008F7D8093B0000895FF9210
:105540000F931F93F62E482F50E0CA01895E934FA8
:10555000FC012491CA018D5F934FFC0114914151CC
:10556000544FFA0104910023C9F0222319F0822F2D
:105570000E94722AE02FF0E0EE0FFF1FE552F44F79
:10558000A591B4919FB7F894FF2021F48C911095C8
:10559000812302C08C91812B8C939FBF1F910F910F
:1055A000FF9008950F931F93482F50E0CA01895E22
:1055B000934FFC012491CA018D5F934FFC0104912C
:1055C0004151544FFA011491112319F420E030E0B5
:1055D00015C0222319F0822F0E94722A812F90E099
:1055E000880F991F8B51944FFC01A591B4918C9118
:1055F00020E030E0802311F021E030E0C9011F916C
:105600000F910895982F8E3008F09E5097708091DA
:1056100048038295880F880F807C892B80937C00BB
:1056200080917A00806480937A0080917A0086FD70
:10563000FCCF2091780040917900942F80E030E0F9
:10564000282B392BC9010895A0E0B0E0EAE2FBE283
:105650000C94C22F7C016B018A01C0E0D0E00FC026
:10566000D6016D916D01D701ED91FC910190F08112
:10567000E02DC7010995C80FD91F01501040011531
:10568000110571F7CE01CDB7DEB7E8E00C94DE2F3F
:10569000EF92FF920F931F93CF93DF937C018B01C7
:1056A000C0E0D0E0F8010F5F1F4F6491662359F00E
:1056B000D701ED91FC910190F081E02DC701099592
:1056C000C80FD91FEFCFCE01CDB7DEB7E6E00C94FF
:1056D000E02FDC01ED91FC910190F081E02D099526
:1056E0000895EF92FF920F931F938C016DE00E943B
:1056F000692B7C01C8016AE00E94692B9C012E0D78
:105700003F1DC9011F910F91FF90EF900895EF92F7
:10571000FF920F931F937C010E94482B8C01C701BD
:105720000E94712B9C01200F311FC9011F910F9105
:10573000FF90EF900895EF92FF920F931F937C01DB
:105740000E94692B8C01C7010E94712B9C01200FC4
:10575000311FC9011F910F91FF90EF900895CF93D2
:10576000DF93EC016115710519F420E030E00FC002
:10577000DB010D900020E9F71197A61BB70BE8811C
:10578000F9810280F381E02DAD0109959C01C901E9
:10579000DF91CF9108954F925F927F928F929F9267
:1057A000AF92BF92CF92DF92EF92FF920F931F932F
:1057B000DF93CF93CDB7DEB7A1970FB6F894DEBFD6
:1057C0000FBECDBF2C01742ECB01223008F42AE08D
:1057D00019A231E2C32ED12CCC0EDD1E822E9924CB
:1057E000AA24BB24672D752FA50194010E947B2F4D
:1057F00079018A01C801B701A50194010E94492FCE
:10580000472D461B0894C108D1084A3010F4405D6A
:1058100001C0495CF6014083E114F1040105110562
:1058200021F07E2C5F2DC801DDCFC201B6010E94A0
:10583000AF2BA1960FB6F894DEBF0FBECDBFCF91B0
:10584000DF911F910F91FF90EF90DF90CF90BF906D
:10585000AF909F908F907F905F904F900895DC0164
:105860002115310541F4ED91FC910190F081E02D7D
:10587000642F099508950E94CB2B0895EF92FF9213
:105880000F931F937C010E942F2C8C01C7010E9453
:10589000712B9C01200F311FC9011F910F91FF90A7
:1058A000EF900895EF92FF920F931F939A017B015F
:1058B00000E010E0B801A7010E942F2C1F910F916A
:1058C000FF90EF900895EF92FF920F931F937C014A
:1058D0000E94522C8C01C7010E94712B9C01200F49
:1058E000311FC9011F910F91FF90EF900895EF9222
:1058F000FF920F931F939A01E62EFF2400E010E021
:10590000B801A7010E942F2C1F910F91FF90EF90DB
:105910000895EF92FF920F931F937C010E94772CC2
:105920008C01C7010E94712B9C01200F311FC901FE
:105930001F910F91FF90EF900895A0E0B0E0E3EA8F
:10594000FCE20C94C22FEC016A017B0121153105A8
:1059500041F4E881F9810190F081E02D642F0995EF
:105960001BC02A303105B1F477FF13C06DE20E94ED
:10597000692B8C0144275527BA014C195D096E0922
:105980007F09CE012AE00E94CB2B9C01200F311F02
:1059900004C02AE00E94CB2B9C01C901CDB7DEB721
:1059A000E8E00C94DE2FEF92FF920F931F937B01A0
:1059B0009A010027F7FC0095102FB801A7010E945B
:1059C0009D2C1F910F91FF90EF900895EF92FF9201
:1059D0000F931F937C010E94D32C8C01C7010E945E
:1059E000712B9C01200F311FC9011F910F91FF9056
:1059F000EF9008950E94AF2B0895EF92FF920F93BE
:105A00001F937C010E94FA2C8C01C7010E94712B0C
:105A10009C01200F311FC9011F910F91FF90EF9042
:105A2000089508951F920F920FB60F9211242F938D
:105A30003F934F938F939F93EF93FF938091C00079
:105A400082FD1DC04091C6002091ED053091EE050C
:105A50002F5F3F4F2F7330708091EF059091F005CD
:105A60002817390771F0E091ED05F091EE05E35547
:105A7000FA4F40833093EE052093ED0502C08091EC
:105A8000C600FF91EF919F918F914F913F912F9180
:105A90000F900FBE0F901F9018951F920F920FB688
:105AA0000F9211242F933F938F939F93EF93FF9324
:105AB0002091310630913206809133069091340660
:105AC0002817390731F48091C1008F7D8093C10080
:105AD00014C0E0913306F0913406EF50FA4F208164
:105AE000809133069091340601968F739070909355
:105AF0003406809333062093C600FF91EF919F9167
:105B00008F913F912F910F900FBE0F901F9018957E
:105B1000A0E0B0E0EEE8FDE20C94BE2FFC011382A1
:105B2000128288EE93E0A0E0B0E084839583A683A0
:105B3000B7838BE893E09183808375876487578769
:105B40004687318B208B138B028BF58AE48AD78AA8
:105B5000C68AB18EA08E938E828E8F85848F88891F
:105B6000858F8989868F8A89878F8B8980A32096E4
:105B7000ECE00C94DA2FAF92BF92DF92EF92FF929B
:105B80000F931F93CF93DF93EC017A018B01DD24F8
:105B9000403081EE580780E0680780E0780711F018
:105BA000DD24D39491E0A92EB12CEC89FD89DD2070
:105BB00069F0C50108A002C0880F991F0A94E2F796
:105BC000808360E079E08DE390E005C0108260E8BA
:105BD00074E88EE190E0A80197010E947B2F21508C
:105BE000304040405040569547953795279580E185
:105BF0002030380720F0DD2011F0DD24D6CFE889F1
:105C0000F9893083EA89FB89208319A2EE89FF890B
:105C1000408121E030E0C9010C8C02C0880F991F3F
:105C20000A94E2F7482B4083EE89FF894081C9013D
:105C30000D8C02C0880F991F0A94E2F7482B40830D
:105C4000EE89FF894081C9010E8C02C0880F991F1F
:105C50000A94E2F7482B4083EE89FF8980810F8CFC
:105C600002C0220F331F0A94E2F7209528232083D5
:105C7000DF91CF911F910F91FF90EF90DF90BF9038
:105C8000AF900895DC011C96ED91FC911D97E05CAE
:105C9000FF4F2191319180819181281B390B2F7306
:105CA0003070C901089585E396E00E94422E892B49
:105CB00011F00E94112D0895DC011C96ED91FC91CC
:105CC0001D97E05CFF4F20813181E054F040DF01FF
:105CD000AE5BBF4F8D919C9111972817390719F42E
:105CE0002FEF3FEF07C08D919C91E80FF91F808146
:105CF000282F30E0C9010895DC011C96ED91FC913C
:105D00001D97E05CFF4F20813181E054F040DF01BE
:105D1000AE5BBF4F8D919C9111972817390719F4ED
:105D20002FEF3FEF10C08D919C911197E80FF91F55
:105D300020818D919C91119701968F73907011968F
:105D40009C938E9330E0C9010895DC0191968C916B
:105D50009197882339F05496ED91FC915597808165
:105D600086FFF9CF91961C920895CF93DF93EC01B3
:105D7000EE85FF85E05CFF4F20813181E054F040EB
:105D80002F5F3F4F2F733070DF01AE5BBF4F8D91A0
:105D90009C91119728173907D1F3E05CFF4F808160
:105DA0009181E054F040E80FF91F6083EE85FF8594
:105DB000E05CFF4F31832083EE89FF89208181E001
:105DC00090E00F8C02C0880F991F0A94E2F7282BED
:105DD000208381E089A3EC89FD89808180648083B0
:105DE00081E090E0DF91CF9108958F929F92AF92E2
:105DF000BF92CF92DF92EF92FF920F931F9300D04A
:105E000000D00F92EDB7FEB7319684E0ADB7BEB7C4
:105E100011968C9383E0818387E0828385E083837E
:105E200081E0848385E396E06DEA75E041EF55E01B
:105E300025EC30E004EC10E0B0ECEB2EF12CA1EC02
:105E4000CA2ED12CF2ECAF2EB12CE6EC8E2E912C7A
:105E50000E94882D0F900F900F900F900F901F9120
:105E60000F91FF90EF90DF90CF90BF90AF909F90F9
:105E70008F900895CF93DF930E94F8290E94C62740
:105E8000C3E5DEE20E94EE112097E1F30E94532E5B
:105E9000F9CF629FD001739FF001829FE00DF11D49
:105EA000649FE00DF11D929FF00D839FF00D749F94
:105EB000F00D659FF00D9927729FB00DE11DF91F40
:105EC000639FB00DE11DF91FBD01CF01112408959D
:105ED00097FB092E07260AD077FD04D086D006D07E
:105EE00000201AF4709561957F4F0895F6F790950C
:105EF00081959F4F0895A1E21A2EAA1BBB1BFD019D
:105F00000DC0AA1FBB1FEE1FFF1FA217B307E40798
:105F1000F50720F0A21BB30BE40BF50B661F771FF0
:105F2000881F991F1A9469F76095709580959095D0
:105F30009B01AC01BD01CF01089597FB092E0526F9
:105F40000ED057FD04D0D7DF0AD0001C38F450958E
:105F50004095309521953F4F4F4F5F4F0895F6F78D
:105F600090958095709561957F4F8F4F9F4F0895C5
:105F70002F923F924F925F926F927F928F929F9259
:105F8000AF92BF92CF92DF92EF92FF920F931F9347
:105F9000CF93DF93CDB7DEB7CA1BDB0B0FB6F894F8
:105FA000DEBF0FBECDBF09942A88398848885F8438
:105FB0006E847D848C849B84AA84B984C884DF80A9
:105FC000EE80FD800C811B81AA81B981CE0FD11D8D
:105FD0000FB6F894DEBF0FBECDBFED010895EE0FF2
:105FE000FF1F0590F491E02D0994AA1BBB1B51E102
:105FF00007C0AA1FBB1FA617B70710F0A61BB70B39
:10600000881F991F5A95A9F780959095BC01CD01DD
:106010000895911106C0803219F089508550D0F74B
:0C6020000895992788270895F894FFCF71
:10602C004E6F005965730054582074696D656F7517
:10603C007421006D6F64756C65206C6F636B6564A7
:10604C003F00486F70206368616E6E656C200020A5
:10605C0040200053004E2F4100386368002C002C68
:10606C00205B005D20280029004E4F5420454E41F6
:10607C00424C45440053656E64696E6720736574C9
:10608C0074696E677320746F2052580A00526573DE
:10609C00657474696E672073657474696E677320B8
:1060AC006F6E2052580A0041626F727465642065ED
:1060BC00646974730A00696E76616C696420736537
:1060CC006C656374696F6E000D0A496E76616C695C
:1060DC006420696E707574202D206469736361721D
:1060EC006465642107007363616E6E6572206D6F69
:1060FC0064650053657474696E67732073617665AB
:10610C006420746F20454550524F4D0A00526576FD
:10611C0065727465642073657474696E6773206648
:10612C00726F6D20454550524F4D0A004C6F6164A3
:10613C00656420666163746F72792064656661754D
:10614C006C74730A004B657920616E64206368611E
:10615C006E6E656C732072616E646F6D697A6564C6
:10616C000A004F70656E4C52536E67205458207362
:10617C0074617274696E672000206F6E204857201E
:10618C000050504D00525353490053444100534367
:10619C004C00525844005458440041494E004C4263
:1061AC004545500053504B54524D005342555300EB
:1061BC0053554D44004C4C494E440000342B340094
:1061CC003800382B340031320031322B3400313668
:1061DC000001000000C01200001A400AA1204EA5C8
:1061EC00001B1E27522C23308025000005400AA1DD
:1061FC00204EA50020244EA52C2330004B00000679
:10620C00400AD0009D49007B289D492C233000E199
:10621C00000005400A4501D7DC03B81E0EBF002361
:10622C002E48E801008A400A6001555502AD1E2037
:10623C00000023C88025000005400AA1204EA500BF
:10624C0020244EA52C233000020002000200020084
:10625C000200020002000200020002000200020022
:10626C0002000200020002FF01610265026A026E76
:10627C0002720276027A027E0284028B02900295EE
:10628C00029B029B029B029B0235019C02A002A274
:10629C0002A602A902AE02350100070B0C10111563
:1062AC0000160A1322312900000000B52E242B42BF
:0862BC002E7C2E5C2EA52E00A5
:107E00000F92CDB7DEB7112484B714BE81FFF1D035
:107E100082E08093C00088E18093C10086E0809377
:107E2000C20080E18093C4008EE0CDD088249924E4
:107E3000CC24C394F5E0DF2EE1E1EE2E73E0F72EC3
:107E4000B6D0082F813479F4B2D08983C2D0898129
:107E5000823811F481E005C0813811F485E001C059
:107E600083E09ED09AC0823411F484E103C085344B
:107E700019F485E0B6D091C0853561F498D0082F0B
:107E800010E095D090E0982E8824802A912A880CC2
:107E9000991C82C0863521F484E0A3D080E0E1CF34
:107EA000843609F04CC083D082D0A82E80D0B82E62
:107EB00000E011E07CD0F80181938F01AE16D1F77C
:107EC00088D0FB2DF53489F4E0E0F1E00BC0F9999E
:107ED000FECF92BC81BC0894811C911C819180BD15
:107EE000FA9AF99AEA1598F358C08B2D863409F05E
:107EF00054C0F401F7BEE89507B600FCFDCFF401CD
:107F0000A0E0B1E02C9130E011968C91119790E0B7
:107F1000982F8827822B932B12960C01C7BEE895C9
:107F20001124329681E0A038B80761F7F401D7BE7A
:107F3000E89507B600FCFDCFE7BEE8952EC0843774
:107F4000F1F435D034D0182F32D0B82E42D0FB2DDA
:107F5000F63421F4F40105914F010CC0FB2DF534EA
:107F600049F4F999FECF92BC81BC0894811C911C04
:107F7000F89A00B5802F14D0115049F70EC08537FC
:107F800039F427D08EE10CD085E90AD08FE069CF93
:107F9000813511F488E017D01CD080E101D050CF9A
:107FA0009091C00095FFFCCF8093C600089580910A
:107FB000C00087FFFCCF8091C00084FD01C0A89560
:107FC0008091C6000895E0E6F0E098E19083808318
:107FD0000895EDDF803219F088E0F5DFFFCF84E10E
:107FE000DFCF1F93182FE3DF1150E9F7F2DF1F9166
:0E7FF0000895282E80E0E7DFEE27FF27099492
:027FFE0001057B
:0400000300007E007B
:00000001FF
